:020000040000FA
:060000000000000087284B
:0800080000000000F0000308F5
:10001000F1000A08F2008C1810280B192528302846
:10002000831203138C1083120313B00B3028B10812
:1000300003191F281930B000B10105113028FA301A
:10004000B0000130B10005153028831203130130D0
:10005000A6070318A70A0B1100008606000000007F
:1000600072088A0071088300F00E700E000009000B
:100070008316031306308600203099002430980040
:100080008312031380309800080083160313981C12
:10009000472883120313340E0F39303E83120313A3
:1000A000990083160313981C5328831203133408F2
:1000B0000F39303E8312031399000800831603138F
:1000C000981C6028831203131B30990083160313B6
:1000D000981C6828831203135B309900831603135E
:1000E000981C70288312031332309900831603136F
:1000F000981C7828831203134A309900831603133F
:10010000981C8028831203130D30990008000730D3
:100110009F0083160313F03085000C3086006400C6
:1001200083166730810083128312031385018601D1
:10013000013083120313B1006A21F12155213820C7
:1001400000000000CD2000000000DC2000000000C6
:10015000000000000F21000000005E2000000000F1
:10016000831203132B08B400452000000000831203
:1001700003132A08B4004520000000008312031373
:100180002908B4004520000000008312031328084A
:10019000B400452000000000A0288312031385113D
:1001A00083160313851183120313A701A601A5016A
:1001B000A4010B1181010800000000008312031349
:1001C0003118E02883120313311CE4281630B200E2
:1001D000B20BE82800000000831603138515831274
:1001E00003133118F12883160313851183120313A7
:1001F0000108A500AE01AE0AAE0803190900851575
:10020000000000000000000000000000851101084F
:1002100025020319FB28AE092E0AA40008000000DD
:1002200000000000C221BD213030AE002C080F3983
:10023000031D1F292B0E0F39031D232927292C08E5
:100240000F392E0795212B0E0F392E0795212B08DC
:100250000F392E0795212E3095212A0E0F392E07A2
:1002600095212A080F392E079521290E0F392E07BF
:1002700095212C30952129080F392E079521280E1C
:100280000F392E07952128080F392E079521203088
:1002900095214D309521483095217A309521203097
:1002A000952120309521BD210800F93083160313D4
:1002B00092004930831203139200FA30B0008B177A
:1002C0000B178B168C10831603138C1483120313D5
:1002D00012150800382285100510303086000514EC
:1002E00000000000051038223030860005140000A0
:1002F000000005104A22303086000514000000007E
:1003000005104A2220308600051400000000051068
:100310004A220C3093214A22063093214A2201308E
:1003200093214F220800851096298514AD00F039DD
:100330008600051400000000000000000000051009
:10034000AA30A000A00BA2292D08F0392D0E86009E
:100350000514000000000000000000000510AA3095
:10036000A000A00BB1290800C03093214A22080048
:10037000013093214F224F220800023093214F2257
:100380004F22080003102030AF00A801A901AA01E4
:10039000AB01AC01A40DA50DA60DA70DA80DA90DCF
:1003A000AA0DAB0DAC0DAF0BD62900342C30840058
:1003B000E6212B308400E6212A308400E621293012
:1003C0008400E62128308400E621CA290330000792
:1003D000AE00AE19800030300007AE00AE1B8000CA
:1003E0000800433095214F309521553095214E30EE
:1003F000952154309521453095215230952120305A
:100400009521203095215630952165309521723007
:10041000952120309521313095212E309521323093
:10042000952119303322B821B42147309521543019
:1004300095213D309521313095212E309521303058
:100440009521203095212030952150309521533031
:1004500095213D309521313095213A30952131302B
:100460009521BD210800A3003822A30B342A0800DF
:100470000930A0005030A1007530A200A20B3E2A26
:10048000A10B3C2AA00B3A2A7730A000A00B462AE9
:1004900000000800A930A000A00B4C2A08000C3076
:1004A000A0008C30A100A10B532AA00B512A0800F8
:1004B00006100000000000008614861008000614D4
:1004C0000000000000000000861486100800803044
:1004D000B3000310330834050319702A5F22722A0F
:0C04E0005822722AB30C031C6A2A080080
:02400E00623F0F
:00000001FF
